S01A000064656D6F70726F675F73746D3332663035312E7372656399
S31508002000D8040020E92A000883230008872300084B
S3150800201000000000000000000000000000000000B2
S31508002020000000000000000000000000072600086D
S315080020300000000000000000C72A0008F927000871
S31508002040D32A0008212B0008232B0008252B00087B
S31508002050272B0008292B00082B2B00082D2B0008FE
S315080020602F2B0008312B0008332B0008352B0008CE
S31508002070372B0008392B00083B2B00083D2B00089E
S315080020803F2B0008412B000800000000432B0008E6
S31508002090452B0008472B0008492B00084B2B000846
S315080020A04D2B00084F2B0008512B0008532B000816
S315080020B0552B000800000000572B00080000000000
S315080020C0EE11AA5530B50400002000250020002195
S315080020D000200025644801680C200840002806D026
S315080020E0042807D0082808D00C2823D025E07048F3
S315080020F0206024E06E48206021E05B480068F025F7
S31508002100AD03054058480168C02040020840AD0CA0
S31508002110AD1C002802D16748454309E066480068B7
S315080021200107090F491C624800F0D4F86843050006
S31508002130256004E06248206001E05D4820604A4866
S315080021400168F020084000095C49085C2168C14024
S31508002150616045480168E020C0000840000A574908
S31508002160085C6168C140A16048480068C00502D49F
S315080021705448E0600AE03C480068400403D4A0687C
S315080021804008E06002E0A0688008E0603F48006818
S31508002190400602D44C48206102E0802000022061FB
S315080021A03A480068C00602D44148606101E02068E8
S315080021B06061364800688007800F002802D1A06851
S315080021C0A0611AE0314800688007800F012802D113
S315080021D02068A06111E02D4800688007800F02285A
S315080021E003D180200002A06107E028480068800724
S315080021F0800F032801D12E48A06124480068C02119
S3150800220089020140002902D1A068E06123E01F4845
S315080022100068C0218902014080204002814202D123
S315080022202068E06117E019480068C021890201406A
S3150800223080208002814203D180200002E0610AE00A
S3150800224012480068C02189020140C02080028142EC
S3150800225001D11748E0610D480068000602D4184805
S31508002260206200E0256230BD0410024000B5C9B204
S31508002270002905D01549096808431449086004E08F
S315080022801249096881431148016000BD30100240B7
S3150800229000B5C9B2002905D00D49096808430C499B
S315080022A0086004E00A49096881430948016000BDDD
S315080022B000127A0000093D002C100240C0000020E0
S315080022C0006CDC02809FD5001280000014100240CA
S315080022D01C1002400022030A8B420BD203098B42D0
S315080022E019D243088B422ED2411A00D201465241D6
S315080022F010467047FF2209023FD012068B4205D3CB
S31508002300121209028B4201D31212090203098B42E7
S3150800231019D300E0090AC3098B4201D3CB01C01ABD
S31508002320524183098B4201D38B01C01A524143099A
S315080023308B4201D34B01C01A524103098B4201D388
S315080023400B01C01A5241C3088B4201D3CB00C01AF5
S31508002350524183088B4201D38B00C01A524143086D
S315080023608B4201D34B00C01A5241884200D3401A0F
S315080023705241CFD201461046704708B500F002F820
S3150800238008BDFEE77047FEE700B5BFF34F8F554817
S3150800239055490860BFF34F8FFEE780B500F009F88E
S315080023A001BD80B500F047F801BD80B5FFF7ECFF29
S315080023B001BD00B589B0012180208002FFF768FFC2
S315080023C0012180208002FFF751FF0122022190207F
S315080023D0C00500F0EAF8012203219020C00500F0AC
S315080023E0E4F80C20009003206946487102206946EB
S315080023F0087100206946887101206946C8716946D6
S315080024009020C00500F07CF8E12000020290002030
S3150800241003900020049000200590002007900C20CF
S31508002420069002A9314800F0EFF801212F4800F084
S315080024304BF909B000BD80B52D480078002813D1A6
S315080024402C4800F03EF801283AD12A48007800289E
S3150800245036D000F0CEF928490860012024490870D2
S315080024600020264908702BE022482449097840189C
S31508002470401C00F026F8012818D120480078401C96
S315080024801E4908701D4800781A490978884217D1EC
S3150800249000201749087017484078FF2810D11548BA
S315080024A0807800280CD1FFF780FF09E000F0A1F939
S315080024B0114909686431814202D200200C4908702A
S315080024C001BD10B504002021084800F01BF90128B9
S315080024D005D1064800F00AF92070012000E0002026
S315080024E010BD00000400FA050CED00E000440040B1
S315080024F029050020D80400201C05002028050020F6
S3150800250070B5002200230024002246E001239340F0
S315080025100C681C409C423FD10B79012B02D00B79E9
S31508002520022B19D183680324150002267543AC4093
S31508002530A343836083684C79150002267543AC4033
S315080025401C438460838801249440A3438380838842
S315080025508C7994401C438480036803241500022662
S315080025607543AC40A343036003680C791500022643
S315080025707543AC401C430460C36803241500022657
S315080025807543AC40A343C360C368CC7915000226E3
S315080025907543AC401C43C460521C102AB6D370BDA8
S315080025A089B28161704701857047F0B40023002322
S315080025B0D2B20B005B075B0F042463439A401300F7
S315080025C089B2CA1004246243821889B2CC10042541
S315080025D06C430419246A0F250E007607760F042724
S315080025E07E43B540AC43146289B2CA1004246243E0
S315080025F08218126A134389B2C9100422514340183B
S315080026000362F0BC7047FEE7F0B589B004000D0020
S315080026100027002600212068012188432060616880
S315080026200800344901400800A9680143616021682F
S315080026300800314901400B006868EA6802432969C5
S31508002640114319432160A16808002C49014008007C
S3150800265069690143A1606846FFF734FD2148844251
S3150800266001D1069E05E02048844201D1079E00E07C
S31508002670029E206800040CD5022070432968FFF7E3
S3150800268029FE07000220464330002968FFF722FE8C
S3150800269008E030002968FFF71DFE070030002968AA
S315080026A0FFF718FE28684008814200D37F1C20687F
S315080026B0000406D578084107490F114838400F002D
S315080026C00743A78109B0F0BD00B5C9B2002904D0F7
S315080026D0016801220A43026003E00168012291436E
S315080026E0016000BD0038014000440040808CC005F0
S315080026F0C00D7047FFCFFFFFF3E9FFFFFFFCFFFFA9
S31508002700F0FF000000B502000020D0690140002952
S3150800271001D0012000E00020C0B200BDF0B540B2F3
S31508002720002821D5374B40B20207120F083A920803
S3150800273004246243334C40B205072D0F083DAD080B
S31508002740042675436459FF258607B60F08277E4376
S31508002750B540AC438901C9B28007800F0825684394
S315080027608140214399501AE0274A40B2830804243D
S315080027706343D258FF238407A40F08256C43A3405C
S315080027809A438901C9B283079B0F0824634399407A
S3150800279011431D4A40B28008042358431150F0BD26
S315080027A080B580214904884201D3012010E0000247
S315080027B0000A401E1549086003210020C043FFF7A0
S315080027C0ADFF002012490860072012490860002062
S315080027D002BD80B510480068FA218900FFF77AFD26
S315080027E0FFF7DEFF002000F001F801BD0B49086085
S315080027F070470A480068704708480068401C07493F
S31508002800086070471CED00E000E400E014E000E01A
S3150800281018E000E010E000E0D000002024050020C9
S3150800282080B53748006801210143354801603548BD
S31508002830006835490140334801603148006833492A
S3150800284001402F4801602E480068314901402C4854
S3150800285001602C4800682F4901402A4801602E482B
S3150800286000680F2188432C4908602C4800682C49C9
S3150800287001402A4801602B480068012188432949FC
S31508002880086000202849086000F001F801BD00B57D
S315080028901120264908601B4800681A49086019482B
S315080028A0006818490860174800682149014015481A
S315080028B0016014480068A02189030143114801609A
S315080028C00F4800688021490401430D4801600C48FF
S315080028D000688001FBD50B48006803218843094935
S315080028E00860084800680221014306480160054857
S315080028F000680C2101400829F9D100BD000000003C
S3150800290000100240041002400CB8FFF8FFFFF6FE64
S31508002910FFFFFBFFFFFFC0FF2C10024030100240F4
S31508002920ACFEFFFF341002400810024000200240AF
S31508002930FF7FC0FF00B583B0012180200003FFF7A9
S3150800294095FC8020800000900120694608710020CF
S315080029506946887103206946487100206946C8712E
S3150800296069461648FFF7CCFD802189001348FFF712
S315080029701AFE07BD10B5FFF73CFF040010480068B3
S31508002980201AFA214900884216D30E4800780028F2
S3150800299008D101200B490870802189000748FFF7F4
S315080029A0FFFD07E0002007490870802189000348D9
S315080029B0FFF7F9FD0248046010BD00000008004852
S315080029C0200500202A05002070B40121002213E00A
S315080029D00468001D0C4202D04D466D1E6419226023
S315080029E0241D1B1F042BFAD225009E0701D5228021
S315080029F0AD1C0B4000D02A700368001D002BE7D1E0
S31508002A0070BC704730B401210268001D002A0FD03F
S31508002A100368C318446808300C4202D04D466D1E40
S31508002A2064191D6825601B1D241D121FECD0F8E7CC
S31508002A3030BC704710B5074979441831064C7C44B8
S31508002A40163404E0081D0A68891888470100A1425F
S31508002A50F8D110BD08000000280000006DFFFFFF38
S31508002A6054000000D80400200000000099FFFFFF72
S31508002A70140000008C000000C000002000000000C8
S31508002A8080B500F007F8FFF788FCFFF773FFFFF73C
S31508002A9088FCFAE780B5FFF74DFFFFF79AFE01BD00
S31508002AA000F00BF8002801D0FFF7C4FF002000BF94
S31508002AB000BFFFF7E5FF00F002F80120704780B578
S31508002AC000F002F801BDFEE70746384600F002F8B6
S31508002AD0FBE7FEE780B500BF00BF024A11001820D9
S31508002AE0ABBEFBE72600020002488546024880473F
S31508002AF002480047D804002021280008152B0008A2
S31508002B000000000001020304010203040607080985
S31508002B10006CDC0200BF00BF00BF00BFFFF7C0FFAC
S31508002B20FEE7FEE7FEE7FEE7FEE7FEE7FEE7FEE76F
S31508002B30FEE7FEE7FEE7FEE7FEE7FEE7FEE7FEE75F
S31508002B40FEE7FEE7FEE7FEE7FEE7FEE7FEE7FEE74F
S30D08002B50FEE7FEE7FEE7FEE7DB
S70508002B15B2
